:10000000782B820700340034013401340234023486
:100010000334033404340534063407340834093413
:100020000A340B340C340E341034123414340F30C0
:10003000831201058207000000000000000000009C
:1000400000000000000000000000000000000000B0
:100050000000000045088500E2308100410884006E
:100060000508C200C30A0008C400840A0008C500CD
:10007000840A4C30841E0408C1004408850008002E
:10008000A2011430220203184B284C3022078400AE
:100090008001A20A41284C30C100C501FC3081001A
:1000A0001728FF2383169000083085008312101054
:1000B0000C1008308316810083121016901610144D
:1000C00019159914191485010800A3000E08B6002B
:1000D00033083602031CB40A3608B3002308360777
:1000E000B5000E083506031D71280800A200B401F2
:1000F00064303402031884282230850022086520E9
:1001000085012208652078280800B4016430340293
:1001100003188D280A30652086280800B301B40131
:100120008E01573076206730762085208520852007
:100130006730762061307620573076203330762055
:10014000852033307620852041307620852085201B
:100150008528A30083128C13220883169B00230892
:100160009A001C1555309D00AA309D009C141C114E
:1001700083128C1FB82883128C1383120800A200EC
:10018000220883169B001C141A08A300831223085C
:1001900008000030BF20B90039082A3A031DD428CE
:1001A0000130BF20B900D828A2012A30A920B90106
:1001B00008001C30BA001C30BB001C30BC001C30D6
:1001C000BD002730BE002730BF002730C000080028
:1001D000BA1B17281720AD080319F0281C30BA00E5
:1001E000BA031720BA1FFD280130A2003908A92040
:1001F00017200A30AB000A30AC00BB1B1B291720AC
:10020000AC1F0629F7302C02031C08291C30BB0048
:100210001720AB1B0F290A302B02031818291720AF
:10022000AB1F1629F7302B02031C18291C30BB000A
:100230001720BB032D291720AB1B25290A302B02C1
:10024000031C2529391417202629391017201C30A2
:10025000BB000A30AB000A30AC001720BC1B4C2995
:100260001720AC1B372909302C02031839291C3000
:10027000BC001720AB1B402909302B020318492969
:100280001720AB1F4729F6302B02031C49291C30CD
:10029000BC001720BC035C291720AB1B5629093072
:1002A0002B02031C5629B91417205729B9101720FF
:1002B0001C30BC00AB01AC011720BD1B6B29172003
:1002C000AD1B662914302D02031868291C30BD00AF
:1002D0001720BD03782917202B08BE072C08BF075D
:1002E0002E08C0071C30BD000A30AB000A30AC003D
:1002F0001720AD0117281720C601C30117200830A9
:100300000505290603199A29C31F7E29C301172051
:1003100008300505290603199A29C31F8729C30137
:10032000172008300505290603199A29C31F9029AB
:1003300017200134C301172008304205290603198C
:10034000C60A172000341720A30104302302031823
:10035000E32917201A30C3021720083005052906A3
:10036000031DB629C31BAC291720013417201A30EE
:100370004307B7001720B71BC02902303702031C00
:100380000134E530C3071720083005052906031995
:10039000CD29C31BC329172001341720343043074C
:1003A000B70017202B302307840037088000023065
:1003B000C3001720B71BDF2919303702031C013493
:1003C0001720A30AA52917202A08033A031DF1299B
:1003D0002D08B70017202E08AD003708AE001720F3
:1003E000003417202A0BFD292C08B70017202D08F0
:1003F000AC003708AD00172000341720AA08031DF1
:100400000F2A2B08B70017202C08AB003708AC00C8
:100410002C08B70017202D08AC003708AD001720B6
:10042000003417202F082B07AF000310AF0C2F0844
:10043000AB00172030082C07B0000310B00C3008B8
:10044000AC00172031082D07B1000310B10C3108A2
:10045000AD00172032082E07B2000310B20C32088C
:10046000AE0017203E08AB023F08AC021E30AD02C2
:100470004008AE021720AD1BAD01E8201720391C43
:10048000472A2B08B7002C08AB023708AC07172007
:10049000AB1F4F2AAB09AB0A0130B300512A02301F
:1004A000B3001720AC1F592AAC09AC0A1030B400B5
:1004B0005B2A2030B4001720AE1F622AAE09AE0AB4
:1004C000B601632AB60117202B08AB072C08AC072E
:1004D0002E08AE071720AB1B732A15302B02031C06
:1004E000732A1430AB001720AC1B7C2A15302C0269
:1004F000031C7C2A1430AC001720AD1B852A153054
:100500002D02031C852A1430AD001720AE1B8E2A45
:1005100015302E02031C8E2A1430AE001720B91C91
:10052000172817202B080120AB0017202C080120CA
:10053000AC0017202E080120AE001728A501A60147
:10054000A701A8011720A3011430230203181728BC
:100550001720A2012B08A502A51FB32A17201430CB
:10056000A5073308A20717202C08A602A61FBD2A3C
:1005700017201430A6073408A20717202D08A70259
:10058000A71FC72A17201430A7073508A20717206E
:100590002E08A802A81FD12A17201430A807360851
:1005A000A20717204C302307840022088000172060
:1005B000A30AA42AAD01B8010430B5000800172031
:1005C0000630C70080300F07C80008001720480811
:1005D0000F028039031D172817208030C807C7086D
:1005E000031D1B2B17200630C7000230AB00013063
:1005F000B3001720391CFF2A0230AC00002BAC01DD
:1006000017201030B4003808AD000230AE00B6013B
:1006100017209E2217200314AD1F03102D0CB700C6
:100620002D08B70717200314B71F0310370CAD00B0
:1006300017202D08B800C7031728172006300F070A
:10064000CA0002300F07C900172049080F0280397D
:100650000319412B1720083005052906031D3F2BE0
:10066000172002300F07C9002908083CA9001720ED
:100670004A080F028039031D3F2B17200134172031
:10068000252B1720003417200230AA0017201D2325
:10069000003A03194D2B1720472B7B21003A031DED
:1006A000462B1720A321003A0319582B1720462B5D
:1006B000B3011720A20104302202031817281720C3
:1006C0002B30220784000008B70017202730B7021C
:1006D000B71F6C2BB709B70A172033083702031C62
:1006E000752B3708B3002208AA001720A20A5B2B3B
:1006F00051208E20C920DA22A001D920A901A10110
:100700000430210203188B2B2F302107840027305F
:100710008000A10A802B40204323A0080319DF2278
:1007200017200430A00017201720A008031DE62280
:1007300017201D23003A031DB62B17207B21003AFA
:10074000031DB62B1720A321003A031DB62B17203B
:1007500011221720A0080319B02BA0031720942BF7
:1007600017209E2217202D08B800942B17208D2BC0
:0207FE000934BC
:044200002A00000090
:02400E00043F6D
:00000001FF
